:100000000C945C000C9479000C9479000C947900A9
:100010000C9479000C9479000C9479000C9479007C
:100020000C9479000C9479000C9479000C9479006C
:100030000C9479000C9479000C9479000C9479005C
:100040000C94DD010C9479000C9479000C947900E7
:100050000C9479000C9479000C9479000C9479003C
:100060000C9479000C947900000000070002010054
:100070000003040600000000000000000102040864
:100080001020408001020408102001020408102002
:10009000040404040404040402020202020203032E
:1000A0000303030300000000250028002B000000CC
:1000B0000000240027002A0011241FBECFEFD8E043
:1000C000DEBFCDBF11E0A0E0B1E0EEE9F5E002C097
:1000D00005900D92AA31B107D9F711E0AAE1B1E07C
:1000E00001C01D92A332B107E1F70E94D0010C9428
:1000F000CD020C940000CF93DF93C4E0D1E088815F
:10010000229661E00E941A0181E0C831D807B9F750
:10011000DF91CF910895AF92BF92CF92DF92EF928D
:10012000FF920F931F93CF93DF938EE00E94D40032
:10013000BC01882777FD8095982F1F921F921F92F0
:100140002AE02F93A12CB12C6501EE24EA9413E050
:10015000F12E00E010E020E030E0A9010E948901CA
:100160007B0104E011E00F900F900F900F90C0E022
:10017000D0E0CE15DF0514F461E001C060E0F801C5
:1001800080810E94530121960E5F1F4FCA30D10516
:1001900081F7DF91CF911F910F91FF90EF90DF904A
:1001A000CF90BF90AF9008958E3008F08E5087703A
:1001B0002091180190E4299F90011124822B8093B3
:1001C0007C0080917A00806480937A0080917A002C
:1001D00086FDFCCF809178002091790090E0922BF1
:1001E0000895833081F028F4813099F08230A1F0B5
:1001F00008958630A9F08730B9F08430D1F4809129
:1002000080008F7D03C0809180008F778093800075
:10021000089584B58F7702C084B58F7D84BD08951D
:100220008091B0008F7703C08091B0008F7D809364
:10023000B0000895CF93DF9390E0FC01E458FF4FA6
:100240002491FC01E057FF4F8491882349F190E00D
:10025000880F991FFC01E255FF4FA591B4918C5571
:100260009F4FFC01C591D4919FB7611108C0F894CC
:100270008C91209582238C93888182230AC06230DE
:1002800051F4F8948C91322F309583238C9388818C
:10029000822B888304C0F8948C91822B8C939FBF0F
:1002A000DF91CF9108950F931F93CF93DF931F9208
:1002B000CDB7DEB7282F30E0F901E859FF4F849120
:1002C000F901E458FF4F1491F901E057FF4F0491F1
:1002D0000023C9F0882321F069830E94F10069811D
:1002E000E02FF0E0EE0FFF1FEC55FF4FA591B4910A
:1002F0009FB7F8948C91611103C01095812301C0C0
:10030000812B8C939FBF0F90DF91CF911F910F9105
:1003100008954F925F926F927F92AF92BF92CF9269
:10032000DF92EF92FF920F931F93CF93DF93CDB79E
:10033000DEB729013A01621B730B840B950B2989E7
:100340003A894B895C892A193B094C095D09298B3B
:100350003A8B4B8B5C8B9B01AC0169897A898B89C9
:100360009C890E946202E418F50806091709A80191
:1003700097010E9472022A0D3B1D4C1D5D1DCA0192
:10038000B901DF91CF911F910F91FF90EF90DF9016
:10039000CF90BF90AF907F906F905F904F900895F7
:1003A0000E9427020E947B00C0E0D0E00E948B00E8
:1003B0002097E1F30E940000F9CF1F920F920FB631
:1003C0000F9211242F933F938F939F93AF93BF93DB
:1003D00080911B0190911C01A0911D01B0911E0103
:1003E00030911A0123E0230F2D3720F40196A11D2F
:1003F000B11D05C026E8230F0296A11DB11D209353
:100400001A0180931B0190931C01A0931D01B093CE
:100410001E0180911F0190912001A0912101B091B6
:1004200022010196A11DB11D80931F01909320010F
:10043000A0932101B0932201BF91AF919F918F9121
:100440003F912F910F900FBE0F901F9018957894A9
:1004500084B5826084BD84B5816084BD85B58260C9
:1004600085BD85B5816085BDEEE6F0E08081816067
:100470008083E1E8F0E01082808182608083808167
:1004800081608083E0E8F0E0808181608083E1EB3F
:10049000F0E0808184608083E0EBF0E08081816027
:1004A0008083EAE7F0E080818460808380818260DD
:1004B00080838081816080838081806880831092C6
:1004C000C1000895DB018F939F930E949102BF9119
:1004D000AF91A29F800D911DA39F900DB29F900D93
:1004E00011240895052E97FB1EF400940E948902A2
:1004F00057FD07D00E949C0207FC03D04EF40C94D9
:10050000890250954095309521953F4F4F4F5F4F51
:10051000089590958095709561957F4F8F4F9F4F6F
:1005200008950E94BE02A59F900DB49F900DA49FB8
:10053000800D911D11240895A1E21A2EAA1BBB1B48
:10054000FD010DC0AA1FBB1FEE1FFF1FA217B3079F
:10055000E407F50720F0A21BB30BE40BF50B661FB5
:10056000771F881F991F1A9469F760957095809579
:1005700090959B01AC01BD01CF010895A29FB001F0
:10058000B39FC001A39F700D811D1124911DB29FC7
:0E059000700D811D1124911D0895F894FFCF68
:10059E000100000002000300040005000600070031
:0A05AE00080009000A000B0001001C
:00000001FF
